:0200000480007A
:100000006F000005732F2034930F80006308FF03F7
:10001000930F90006304FF03930FB0006300FF038E
:10002000130F000063040F0067000F00732F2034CC
:1000300063540F006F00400093E19153171F0000BD
:1000400023223FFC171F000023200FFC6FF01FFF2F
:100050009300000013010000930100001302000050
:100060009302000013030000930300001304000038
:100070009304000013050000930500001306000020
:100080009306000013070000930700001308000008
:10009000930800001309000093090000130A0000F0
:1000A000930A0000130B0000930B0000130C0000D8
:1000B000930C0000130D0000930D0000130E0000C0
:1000C000930E0000130F0000930F0000732540F102
:1000D0006310050097020000938202017390523072
:1000E000735044749702000093820201739052305F
:1000F00073500018970200009382020273905230EE
:10010000B70200809382F2FF7390023B9302F001EA
:100110007390023A7350403097020000938242017C
:100120007390523073502030735030309301000080
:1001300097020000938242ED739052301305100035
:100140001315F501634C05000F00F00F930110002B
:100150009308D0051305000073000000930200000F
:10016000638A020073905210B7B20000938292101B
:100170007390223073500030970200009382420146
:1001800073901234732540F17300203093012000E6
:10019000370500809305008097260000938686E649
:1001A00023A0A6002FA7B680B7030080631A7706A6
:1001B0009301300083A70600B7030080639277069F
:1001C000930140009305F0FF23A006002FA7B680FF
:1001D00093030000631677049301500083A7060081
:1001E0009303F0FF639E77029301600013051000F4
:1001F000B7050080972600009386C6E023A0A600DE
:100200002FA7B68093031000631C77009301700042
:1002100083A70600B7030080639477006310300261
:100220000F00F00F638001009391110093E1110022
:100230009308D00513850100730000000F00F00F34
:10024000930110009308D00513050000730000000F
:10025000731000C00000000000000000000000005B
:10026000000000000000000000000000000000008E
:0C02700000000000000000000000000082
:1010000000000000000000000000000000000000E0
:1010100000000000000000000000000000000000D0
:1010200000000000000000000000000000000000C0
:1010300000000000000000000000000000000000B0
:081040000000000000000000A8
:040000058000000077
:00000001FF
